:1000000012C02CC02BC0FEC591C528C027C026C079
:1000100025C024C023C022C021C020C01FC01EC0D4
:100020001DC01CC01BC011241FBECFE5D4E0DEBF25
:10003000CDBF10E0A0E6B0E0E4E2FAE102C0059036
:100040000D92AC3BB107D9F710E0ACEBB0E001C0CA
:100050001D92A13FB107E1F7B2DAE2CCD1CF969879
:1000600097988E988F9808958E9A82E08A95F1F7E6
:1000700008958F9A82E0982F9A95F1F78E98982F8D
:100080009A95F1F78F98982F9A95F1F78E9A8A950D
:10009000F1F708958F9A8E9A82E0982F9A95F1F74A
:1000A0008F98982F9A95F1F78E988A95F1F7089581
:1000B00020E042E08F9A87FF02C08E9801C08E9A9E
:1000C00032E0942F9A95F1F78F98942F9A95F1F743
:1000D0002F5F283011F0880FEDCF8F9A8E98832FE5
:1000E0008A95F1F78F98832F8A95F1F780B38295DF
:1000F00086958695837080FD02C080E008958FEF1D
:100100000895482F8F9A8E9882E0982F9A95F1F74C
:100110008F988A95F1F720B3229526952695217020
:1001200090E032E08F9A832F8A95F1F78F98832F92
:100130008A95F1F7220F869921609F5F973091F79A
:100140008F9A442311F48E9A01C08E9882E0982FE2
:100150009A95F1F78F988A95F1F7822F08950F936A
:100160001F93880F413071F4162F180F02E005C05D
:1001700091DF8E9A802F8A95F1F7812F99DF8F3F3B
:10018000B9F302C0860F94DF1F910F910895DC012F
:1001900020E040E050E098E115C0FD01E40FF51FBC
:1001A000E08138E08E2F8227F82FF17080FD29271B
:1001B0002695F13009F42068315011F0E695F2CF20
:1001C0004F5F5F4F4617570741F7822F0895DC01B5
:1001D000CB0181159105A105B10529F08150904011
:1001E000A040B040D9F70895282F30E02077307034
:1001F000A90173E0440F551F7A95E1F7220F331FD1
:10020000420F531F94E0559547959A95E1F78F70EB
:10021000840F0895E82FF0E040E050E08E2F6AE070
:10022000B7DB292F8E2FB4DBE82F30E0042E02C07D
:10023000220F331F0A94E2F7F22B4C5F5F4F4031DD
:10024000510561F78F2F08950F931F93182F062FD5
:100250000BDF80ED2DDF812F2BDF802F29DF1ADFD1
:100260001F910F910895FF920F931F93182F062F40
:10027000F42EFADE80ED1CDF84E01ADF812FCADF66
:1002800017DF802FC7DF14DF8F2DC4DF11DF02DF00
:100290001F910F91FF900895FF920F931F93F82ED7
:1002A000062F142FE1DE80ED03DF80E001DF812FD8
:1002B000B1DFFEDE802FAEDFFBDE8F2DABDFF8DEA1
:1002C000E9DE1F910F91FF9008951F93182F13706F
:1002D0006111106141111068C7DE80EDE9DE87E031
:1002E000E7DE812FE5DED6DE1F9108951F93182FDC
:1002F000BBDE80EDDDDE812FDBDEB6DE81EDD8DE1C
:1003000080E0FFDE182FC6DE812F1F910895CF9267
:10031000DF92EF92FF920F931F938C017B016A0192
:10032000A3DE80EDC5DE84E0C3DEB4DE9DDE81EDBC
:10033000BFDE81E0E6DE282F30E020773070A901B3
:1003400073E0440F551F7A95E1F7220F331F420FD8
:10035000531F94E0559547959A95E1F78F70840F58
:10036000F801808397DE80DE81EDA2DE81E0C9DEC8
:10037000282F30E020773070A90103E0440F551F8B
:100380000A95E1F7220F331F420F531FB4E0559532
:100390004795BA95E1F78F70840FF70180837ADE75
:1003A00063DE81ED85DE81E0ACDE282F30E0207752
:1003B0003070A901A3E0440F551FAA95E1F7220F61
:1003C000331F420F531FE4E055954795EA95E1F737
:1003D0008F70840FF60180835DDE1F910F91FF9077
:1003E000EF90DF90CF900895CF92DF92EF92FF923F
:1003F0000F931F936C017B018A0136DE80ED58DE7E
:1004000080E056DE47DE30DE81ED52DE81E079DECF
:10041000282F30E020773070A90173E0440F551F7A
:100420007A95E1F7220F331F420F531F94E0559541
:1004300047959A95E1F78F70840FF80180832ADE43
:1004400013DE81ED35DE81E05CDE282F30E02077A1
:100450003070A90103E0440F551F0A95E1F7220F00
:10046000331F420F531FB4E055954795BA95E1F7F6
:100470008F70840FF70180830DDEF6DD81ED18DECD
:1004800081E03FDE282F30E020773070A901A3E023
:10049000440F551FAA95E1F7220F331F420F531F38
:1004A000E4E055954795EA95E1F78F70840FF601E2
:1004B0008083F0DD1F910F91FF90EF90DF90CF9040
:1004C0000895FF920F931F93CF93DF93F82EFB01B4
:1004D000DA01E9018081482F50E0918180E0482BCA
:1004E000592B80E1F81671F4CA018E7F33E0880F32
:1004F000991F3A95E1F726814CE050E0421B5109E3
:10050000480F591F57FF06C081E08C9350954195C5
:100510005F4F01C01C9288E2F81691F48481682F25
:1005200070E0CB01807690708036910549F066FFCF
:1005300002C04E7F05C065FF02C04C7F01C0487FEE
:10054000CA0124E0969587952A95E1F78883842F40
:100550008F70F801808380E0DF91CF911F910F9120
:10056000FF9008950F931F93DF93CF93CDB7DEB71E
:1005700028970FB6F894DEBF0FBECDBF082F162FF9
:10058000DE011196E0E6F0E088E001900D928150E6
:10059000E1F7242F30E081E792E0BC01269FC00103
:1005A000279F900D369F900D112468EE73E010DAAE
:1005B000CB012AE0129FB0011124680F791F00239C
:1005C00079F4FE0131969E01275F3F4F80814817E5
:1005D00019F46F5F7F4F04C03196E217F307B1F74C
:1005E000CB0128960FB6F894DEBF0FBECDBFCF91DA
:1005F000DF911F910F910895882319F070956195EF
:100600007F4F442319F0309521953F4F62177307B0
:1006100014F48FEF089580E0261737070CF481E07B
:100620000895CF93DF93EC01A2D870D8882311F4FA
:1006300081E009C088EBBE0191D960E27EE480E0F0
:1006400090E0C5DD80E0DF91CF9108951F93CF93B7
:10065000DF93182FEB018BD859D8882311F482E04F
:1006600007C084E4BE017AD9113009F058D880E07F
:10067000DF91CF911F9108951F93CF93DF93182F90
:10068000EB0175D843D8882311F482E00FC088E4C9
:10069000BE0164D9113009F042D860E27EE480E006
:1006A00090E095DD113009F04DD880E0DF91CF91D9
:1006B0001F9108950F931F93CF93DF93EC018B014C
:1006C00056D824D8882311F481E00FC08EEBBE01E8
:1006D00045D9C0E0D0E0F8D8F801EC0FFD1F8083C9
:1006E0002196C930D105B9F780E0DF91CF911F91F4
:1006F0000F910895FF920F931F93CF93DF93EC0117
:10070000162F042FF22E33D801D8882311F481E05C
:100710000DC08EE4BE0122D9812FC6D8802FC4D847
:100720008881883211F48F2DBFD880E0DF91CF917E
:100730001F910F91FF9008957F928F929F92AF9299
:10074000BF92CF92DF92EF92FF920F931F93DF93AE
:10075000CF93CDB7DEB729970FB6F894DEBF0FBEA3
:10076000CDBF782E6B015A0149018EEB60E070E03D
:10077000F5D88E010F5F1F4F4AE0E42EF12CEC0EEE
:10078000FD1EA2D8F80181938F01EE15FF05C9F770
:100790007E010894E11CF11CC70169E070E0F7DC00
:1007A000882311F083E007C0872DB701A6019501CA
:1007B000840187DE80E029960FB6F894DEBF0FBE75
:1007C000CDBFCF91DF911F910F91FF90EF90DF9000
:1007D000CF90BF90AF909F908F907F9008956F9231
:1007E0007F928F929F92AF92BF92CF92DF92EF92C1
:1007F000FF920F931F93DF93CF93CDB7DEB7299767
:100800000FB6F894DEBF0FBECDBF6C015B014A018D
:100810003901ADD78EEBB601A1D88E010F5F1F4F06
:100820005AE0E52EF12CEC0EFD1E4ED8F801819316
:100830008F01EE15FF05C9F77E010894E11CF11C3C
:10084000C70169E070E0A3DC882311F083E008C0F1
:10085000F6018081B701A5019401830132DE80E0B9
:1008600029960FB6F894DEBF0FBECDBFCF91DF91B2
:100870001F910F91FF90EF90DF90CF90BF90AF90BE
:100880009F908F907F906F9008950F931F938C018E
:100890006ED784EBB80162D881E0C4D7182F67D730
:1008A000111111E0812F1F910F9108950F931F9344
:1008B000CF93DF938C01EB01F8018081BE0107D853
:1008C000F801808381508D3F28F48881883211F0AF
:1008D000803191F7DF91CF911F910F910895282FCB
:1008E000362F8091C0008823A1F5822F6AE050D86E
:1008F0008093C500822F4CD89093C600832F48D890
:100900008093C700832F44D89093C800842F40D889
:100910008093C900842F3CD89093CA0020E030E037
:1009200041E0F901E658FF4F9081F901EB53FF4F89
:100930008081F901EF52FF4F891711F0408301C008
:1009400010822F5F3F4F2630310559F71092C100BA
:1009500008951092D1001092D2001092D3001092FC
:10096000D4001092D5001092D60008950F931F93D3
:10097000CF93DF93282F362F6AE00AD88093C500E3
:10098000822F06D89093C600832F02D88093C70089
:10099000832FFED79093C800842FFAD78093C90085
:1009A000842FF6D79093CA0020E030E002E013E0F5
:1009B00068EC70E0F901EB53FF4F4081F901E65814
:1009C000FF4F8081841720F4F901EF52FF4F00831D
:1009D000F901E658FF4F8081481720F4F901EF52E2
:1009E000FF4F108350E0E901CF52DF4FD901A658E5
:1009F000BF4F8881823031F48C91841719F08C912B
:100A00008F5F8C938881833031F48C91841719F037
:100A10008C9181508C938C91841751F08CEB92E0E7
:100A2000FB013197F1F70197D9F75F5F593009F76B
:100A30002F5F3F4F2630310509F0BCCFDF91CF91BA
:100A40001F910F9108950F931F93CF93DF93EC01A4
:100A500025E030E06AE048EC50E080917B00809334
:100A60007A0080917C0080937B0080917D00809350
:100A70007C0080917E0080937D0080917F00809338
:100A80007E00F901E658FF4F608388EE93E0FA019B
:100A90003197F1F70197D9F7215030402223E9F639
:100AA0008AE080937A00CE0164E670E07DD7062F5D
:100AB000CE016AE070E078D7CB016AE070E074D7CD
:100AC000182FCE016AE070E06FD725E030E09AE0A1
:100AD00068EC70E0F901E658FF4F0083F901E55832
:100AE000FF4F1083F901E458FF4F8083F901E35869
:100AF000FF4F908348EE53E0FB013197F1F74150EF
:100B00005040D1F7215030402130310519F7809104
:100B1000BA00813031F48091860080937300109286
:100B20007A00DF91CF911F910F9108951F920F923C
:100B30000FB60F9211242F933F934F935F938F9390
:100B40009F93AF93BF93CF93DF93EF93FF9315BA28
:100B500094989398E091C200F0E0ED58FF4F8081A7
:100B600083BD4091C1004931E0F58091C3008F5FA2
:100B70008093C3008231A9F51092C3005091850083
:100B800020E030E0842F90E0EC01C056DF4FDC0124
:100B9000A957BF4FF901EF52FF4F8081813011F00B
:100BA000442349F4F901ED58FF4F513011F48C9171
:100BB00001C0888180834C3061F48091C00088231B
:100BC00041F4F901EB53FF4F8081F901E658FF4FE3
:100BD00080832F5F3F4F26303105E1F64F5F409312
:100BE000C100FF91EF91DF91CF91BF91AF919F91A4
:100BF0008F915F914F913F912F910F900FBE0F906A
:100C00001F9018951F920F920FB60F9211242F93D9
:100C10003F934F938F939F93EF93FF934091C20025
:100C20004630A8F4242F30E0F901E658FF4FE08168
:100C3000F0E0E859FF4F808188BB81E090E0042E0E
:100C400002C0880F991F0A94E2F785BB08C046309E
:100C500031F480918400813011F4949A939A842F16
:100C60008F5F8093C200873010F01092C200FF9116
:100C7000EF919F918F914F913F912F910F900FBEC8
:100C80000F901F9018958091BE00882319F18091D4
:100C9000C0008330F8F42091CF00822F6AE078D62C
:100CA00080937A00822F74D690937B002091D80095
:100CB000822F6ED680937C00822F6AD690937D001F
:100CC0002091CE00822F64D680937E00822F60D642
:100CD00090937F008091BE00882319F18091C0001D
:100CE0008330F8F02091D700822F6AE051D68093AC
:100CF0007A00822F4DD690937B002091E900822FBD
:100D000047D680937C00822F43D690937D0020911C
:100D1000D000822F3DD680937E00822F39D69093CB
:100D20007F008091C000833009F477C0843030F4B4
:100D3000813059F0823009F02BC13BC0843009F476
:100D4000AEC0853009F024C1ECC0819912C08091F9
:100D5000CF008F5F8093CF00883110F01092CF00CA
:100D600088EE93E028EC30E0F9013197F1F7019734
:100D7000D9F7829915C08091CF0081508093CF0020
:100D8000829905C0882319F487E18093CF0088EE0B
:100D900093E028EC30E0F9013197F1F70197D9F7AA
:100DA000B09904C0829B02C0819973C02091CF008A
:100DB00066C0819912C08091D8008F5F8093D8005F
:100DC0008C3310F01092D80088EE93E028EC30E0DD
:100DD000F9013197F1F70197D9F7829915C0809100
:100DE000D80081508093D800829905C0882319F4D7
:100DF0008BE38093D80088EE93E028EC30E0F90193
:100E00003197F1F70197D9F7B09904C0829B02C0DE
:100E1000819981C02091D80074C0819913C08091BC
:100E2000D7008F5F8093D700803218F081E08093E5
:100E3000D70088EE93E028EC30E0F9013197F1F724
:100E40000197D9F7829913C08091D7008150809380
:100E5000D700882319F48FE18093D70088EE93E0C0
:100E600028EC30E0F9013197F1F70197D9F7B09903
:100E700004C0829B02C081990CC02091D700822FB0
:100E80006AE086D580937A00822F82D590937B008A
:100E900008958AE080937A0080937B000895819979
:100EA00013C08091E9008F5F8093E9008D3018F0C6
:100EB00081E08093E90088EE93E028EC30E0F901CE
:100EC0003197F1F70197D9F7829913C08091E90022
:100ED00081508093E900882319F48CE08093E90025
:100EE00088EE93E028EC30E0F9013197F1F70197B3
:100EF000D9F7B09904C0829B02C081990CC020919F
:100F0000E900822F6AE044D580937C00822F40D58F
:100F100090937D0008958AE080937C0080937D000B
:100F2000089581990EC08091D0008F5F8093D0008A
:100F300088EE93E028EC30E0F9013197F1F7019762
:100F4000D9F782990EC08091D00081508093D00053
:100F500088EE93E028EC30E0F9013197F1F7019742
:100F6000D9F7B09904C0829B02C081990CC020912E
:100F7000D000822F6AE00CD580937E00822F08D5A6
:100F800090937F0008958AE080937E0080937F0095
:100F9000089587ED90E069EE70E040ED50E0B7D93C
:100FA0008091860080937300809374008093750015
:100FB0008093760080937700809378008091D700AB
:100FC0006091E9004091D000D1DC08958FEC90E071
:100FD00068ED70E04EEC50E007DA8091CF00609150
:100FE000D8004091CE007BDC089580917A00882360
:100FF00051F520E030E06AE048EC50E080917E005E
:1010000080937F0080917D0080937E0080917C00A2
:1010100080937D0080917B0080937C0080917A009A
:1010200080937B00F901E658FF4F608388EE93E0E0
:10103000FA013197F1F70197D9F72F5F3F4F26302B
:101040003105E1F625C020E030E06AE048EC50E0F0
:1010500080917E0080937F0080917D0080937E0050
:1010600080917C0080937D0080917B0080937C0048
:10107000F901E658FF4F608388EE93E0FA0131975B
:10108000F1F70197D9F72F5F3F4F2430310501F772
:101090008FEC90E068ED70E04EEC50E0A5D9209127
:1010A000CF00822F6AE074D48093C500822F70D461
:1010B0009093C6002091D800822F6AD48093C700F5
:1010C000822F66D49093C8002091CE00822F60D4E6
:1010D0008093C900822F5CD49093CA00AAECB0E040
:1010E00028EC30E080917E0080937F0080917D002D
:1010F00080937E0080917C0080937D0080917B00B6
:1011000080937C0080917A0080937B008C91809307
:101110007A0088EE93E0F9013197F1F70197D9F75A
:10112000119780E0A43CB807E9F608950F931F9348
:101130008C0180918600809373008093740080936B
:10114000750080937600809377008093780081E02B
:1011500060E070E07BDA07521F4FF80180818093D6
:10116000CB006AEB70E049EB50E02DEC30E0E4DAC4
:10117000882331F08FEF8093B90081E08093BA002B
:101180008091BA006091B9004091CD00EBD95BDC51
:101190001F910F910895819926C08091C0008823E6
:1011A00029F48091BF008F5F8093BF008091BF00C2
:1011B0008A3079F480918400813019F4109284008F
:1011C00003C081E0809384006091840080E090E01F
:1011D0001AD488EE93E028EC30E0F9013197F1F76A
:1011E0000197D9F71BC08091BF008823A9F0809197
:1011F000BF008A3088F48AE08093C000CADE80E2B3
:101200009EE428EC30E0F9013197F1F70197D9F726
:101210001092C0001092BF001092BF00829929C0A6
:101220008091C000882329F58AE08093C0008091D6
:10123000CC00882319F080E090E078DF80E29EE423
:1012400028EC30E0F9013197F1F70197D9F7809157
:10125000CC00823061F481E090E068DF80E29EE4BF
:1012600028EC30E0F9013197F1F70197D9F71092A6
:10127000C00080995CC08091BE008F5F8093BE00EB
:101280008091C000823031F48091CF006091D8000D
:1012900040E002D88091BE00813049F48091C000C6
:1012A000882329F08091C0008F5F8093C0008091D7
:1012B000BE008A30A9F48091C000882389F481E0BF
:1012C0008093C0001092840080ED97E028EC30E01D
:1012D000F9013197F1F70197D9F781E08093840004
:1012E0008091C0008630C8F01092840088EE93E0B0
:1012F00028EC30E0F9013197F1F70197D9F781E057
:10130000809384008091D7006091E9004091D000E3
:10131000AAD71092C0001092BE0088EE93E028EC8D
:1013200030E0F9013197F1F70197D9F708958091ED
:10133000C000882399F58091BE00882379F18091BF
:1013400083008F5F809383001092BD0080918300A3
:10135000843010F0109283009AE09093C000909334
:101360007A0010927B00809183008F5F80937C00D5
:1013700090937D0090937E0090937F0088E893E1A6
:1013800028EC30E0F9013197F1F70197D9F7109285
:10139000C0006091830081E090E035D31092BE00E0
:1013A000089580918300813051F0813030F0823097
:1013B00021F1833009F0A3C055C008DE50C08091F0
:1013C000BD00893708F402DE8091BD00893709F439
:1013D000E0DD8091BD00833808F491C08FEC90E08F
:1013E00068ED70E04EEC50E0FFD78091CF00609147
:1013F000D8004091CE00BADA32C08091BD00893762
:1014000008F4E4DD8091CC00882371F0813071F420
:101410008091BD00893719F480E090E087DE8091EB
:10142000BD00833818F0E1DD1092BD008091CC0042
:10143000823009F064C08091BD00893719F480E0E2
:1014400090E074DE8091BD00833819F481E090E073
:101450006DDE8091BD008D3808F451C0C6DD10925C
:10146000BD0008958091BD00893708F4AFDD8091FB
:10147000BD00893709F48DDD8091CC008823A1F46B
:101480008091BD00833880F08FEC90E068ED70E0D3
:101490004EEC50E0A9D78091CF006091D8004091E8
:1014A000CE0064DA1092BD008091CC00813071F4DE
:1014B0008091BD00833819F480E090E037DE8091A0
:1014C000BD008D3818F091DD1092BD008091CC00E8
:1014D0008230A9F48091BD00833819F480E090E057
:1014E00025DE8091BD008D3819F481E090E01EDE8C
:1014F0008091BD00873918F078DD1092BD00089505
:101500008F929F92AF92BF92DF92EF92FF920F93D2
:101510001F93DF93CF93CDB7DEB729970FB6F8941B
:10152000DEBF0FBECDBF8FEF898300E010E022E069
:10153000E22EF12CEC0EFD1E4E010894811C911C34
:101540009AE0A92EB12CAC0EBD1E1FC0C401B7017C
:10155000ADD989818F3F19F08E3F39F48FEF809399
:10156000B90081E08093BA0017C0D701F80183E089
:10157000EE0FFF1F8A95E1F7E752FF4F8D918193A0
:10158000AA15BB05D9F70F5F1F4FD02E898188237D
:1015900019F002301105D1F68D2D29960FB6F89469
:1015A000DEBF0FBECDBFCF91DF911F910F91FF9096
:1015B000EF90DF90BF90AF909F908F900895EF9243
:1015C000FF920F931F9384B38F6384BB87B38C63A5
:1015D00087BB81B3886181BB85B5836085BD89B7D1
:1015E000806C89BF3CD580E061E041E06ED680E34D
:1015F00090E062E370E041E350E025E0FCD080DF62
:101600008093CC00882321F081E060E070E01ED858
:1016100088EE93E028EC30E0F9013197F1F701977B
:10162000D9F782E090E0E7D1813061F080E090E08E
:1016300061E0E9D181E090E063E0E5D182E090E013
:1016400061E0E1D180E090E0D6D18093840081E038
:1016500090E0D1D18093830078949AE09093C00079
:1016600090937A0010927B00809183008F5F80932B
:101670007C0090937D0090937E0090937F0080E2A9
:101680009EE428EC30E0F9013197F1F70197D9F7A2
:101690001092C00087ED90E069EE70E040ED50E000
:1016A00036D6EE24E3941AE039E6F32E08EC809166
:1016B000C0008111E8DA6FDDB09B25C08091C000C9
:1016C000882309F58091BC00882389F78091BC00AC
:1016D0008F5F8093BC008091BD008F5F8093BD00C1
:1016E0008091CF00873038F410928500F092860008
:1016F0000093790006C0E092850010938600109355
:1017000079004FDED4CF1092BC00D1CFE091ED0034
:10171000F091EE0080819091EC0089230895E09192
:10172000EA00F091EB0080819091EC00892B80839E
:10173000E091EF00F091F00080819091EC00892B16
:1017400080830895E091EA00F091EB009081809110
:10175000EC00809589238083E091EF00F091F00008
:1017600090818091EC008095892380830895E09199
:10177000EA00F091EB0090818091EC008095892344
:101780008083E091EF00F091F00080819091EC0077
:10179000892B808385EA95E08115910511F00197E9
:1017A000F1F72FB7F894E091EF00F091F0009081FD
:1017B0008091EC0080958923808386EC90E08115F0
:1017C000910511F00197F1F7E091ED00F091EE0035
:1017D00040813091EC002FBF8EED94E08115910592
:1017E00011F00197F1F78081832311F481E00895CE
:1017F000842F832308955093F0004093EF0070935B
:10180000EB006093EA009093EE008093ED0081E09E
:1018100090E002C0880F991F2A95E2F78093EC00B0
:10182000A6DF0895382F4FB7F894E091EF00F091BC
:10183000F00080819091EC00892B808382E090E021
:101840008115910511F00197F1F7332351F0E091E3
:10185000EF00F091F00090818091EC008095892359
:10186000808386E290E08115910511F00197F1F7F0
:10187000E091ED00F091EE0080812091EC00822358
:1018800009F430E087E890E08115910511F00197A7
:10189000F1F7E091EF00F091F0008081209528238E
:1018A00020834FBF832F08950F931F93182F08E0B5
:1018B000812F8170B7DF1695811110680150C1F733
:1018C000812F1F910F9108958FEFEEDF0895DF9222
:1018D000EF92FF920F931F93CF93DF93E82EEB01CC
:1018E00046DF882381F580EFDFDF80E4FF24182FB7
:1018F00098EFD92ED80E81E095DF082F81E092DF96
:10190000882329F0002371F08EEFF82E1EC00023EB
:1019100049F41E1528F0888180FF04C0E11611F0FB
:10192000F12E01E0802F7EDF888186958883002359
:1019300011F08068888311501D15E9F6112329F0F4
:101940002196812FD4CFFF24FA948F2DDF91CF9150
:101950001F910F91FF90EF90DF9008950F931F93C9
:10196000CF93DF93082FEB0102DF209741F085E54D
:101970009BDF18E0899198DF1150E1F702C08CECF1
:1019800093DF802F91DFDF91CF911F910F91089509
:10199000991B79E004C0991F961708F0961B881FC1
:1019A0007A95C9F780950895AA1BBB1B51E107C022
:1019B000AA1FBB1FA617B70710F0A61BB70B881FDF
:1019C000991F5A95A9F780959095BC01CD0108956E
:1019D00097FB092E07260AD077FD04D0E5DF06D055
:1019E00000201AF4709561957F4F0895F6F7909551
:1019F00081959F4F0895E199FECF9FBB8EBBE09AE2
:101A000099278DB30895262FE199FECF9FBB8EBBFA
:101A10002DBB0FB6F894E29AE19A0FBE0196089595
:041A2000F894FFCF68
:101A240001030406090B0C0E002010300828183896
:101A340004243CFF0101FFFFFFFF0A0A0A0A0A0A05
:101A4400000000020101FA01152A3F54697E93A89F
:101A5400BDD2E7F5E7D2BDA8937E69543F2A1501AC
:101A640069747F8A95A2AFBAC6D2DEEAF5EADED2FD
:0C1A7400C6BAAFA2958A7F7469FF01001A
:00000001FF
